:020000040800F2
:1000000000060020E1010008E3010008E301000808
:10001000E3010008E3010008E3010008E301000830
:10002000E3010008E3010008E301000801360008CD
:10003000E3010008E3010008E3010008E301000810
:10004000E3010008E3010008E3010008E301000800
:10005000E3010008E3010008B1380008D9380008BE
:10006000013900082939000851390008E301000866
:10007000E3010008E3010008E3010008E3010008D0
:10008000E3010008E3010008E3010008E3010008C0
:10009000E3010008E3010008E301000879390008E2
:1000A000E3010008E3010008E3010008E3010008A0
:1000B000E3010008E3010008E3010008E301000890
:1000C000E3010008E3010008E3010008E301000880
:1000D000E3010008E30100084D3A0008E3010008CD
:1000E000DD390008E3010008E3010008E30100082E
:1000F000E3010008E3010008E3010008E301000850
:10010000E3010008E3010008613A0008E301000888
:10011000E3010008E3010008E3010008E30100082F
:10012000E3010008E3010008E3010008E30100081F
:10013000E3010008E3010008E3010008E30100080F
:10014000E3010008E3010008E3010008A92D00080D
:10015000E3010008E3010008E3010008E3010008EF
:10016000E3010008E3010008E3010008E3010008DF
:10017000E3010008E3010008E3010008E3010008CF
:10018000E3010008E3010008E3010008E3010008BF
:10019000E3010008E3010008E3010008E3010008AF
:1001A000E3010008E3010008E3010008E30100089F
:1001B000E3010008E3010008E3010008E30100088F
:1001C000E3010008E3010008E3010008E30100087F
:1001D000E3010008E3010008E3010008E30100086F
:1001E00002E000F000F8FEE772B6374880F30888B6
:1001F000364880F3098836483649086040F20000E6
:10020000CCF200004EF63471CEF200010860BFF36C
:100210004F8FBFF36F8F40F20000C0F2F0004EF638
:100220008851CEF200010860BFF34F8FBFF36F8F8C
:100230004FF00000E1EE100A4EF63C71CEF20001E4
:100240000860062080F31488BFF36F8F02F074FA01
:1002500003F074F94FF055301F491B4A91423CBFDF
:1002600041F8040BFAE71D49184A91423CBF41F896
:10027000040BFAE71A491B4A1B4B9A423EBF51F83E
:10028000040B42F8040BF8E700201849184A914281
:100290003CBF41F8040BFAE702F052FA03F0A2F96E
:1002A000144C154DAC4203DA54F8041B8847F9E7A7
:1002B00000F042F8114C124DAC4203DA54F8041B22
:1002C0008847F9E702F03ABA000600200022002031
:1002D0000000000808ED00E00000002000060020FB
:1002E000A03E0008002200204C22002050220020C6
:1002F00020310020E0010008E0010008E0010008D2
:10030000E00100082DE9F04F2DED108AC1F80CD066
:10031000C3689D46BDEC108ABDE8F08F002383F3CF
:1003200011882846A047002001F098FDFEE701F063
:1003300027FD00DFFEE7000038B500F0DFFB02F02C
:10034000CFF940B1164B6FF03F01002259720F21D7
:100350001A729972DA7202F0A9F9054602F0E2F90E
:100360000446C8B90F4B9D4218D001339D4218BFB7
:10037000044641F2883504BF01240025002002F024
:100380009FF90CB100F076F800F018FD284600F057
:10039000C1F800F06FF8F9E70025EFE70546EDE753
:1003A00000220020010007B008B500F073FBA0F1A7
:1003B00020035842584108BD07B541F212030221FB
:1003C00001A8ADF8043000F083FB03B05DF804FB36
:1003D00038B5302383F31188174803680BB101F057
:1003E00009FE164A144800234FF47A7101F0F8FD13
:1003F000002383F31188124C236813B12368013B57
:100400002360636813B16368013B63600D4D2B7813
:1004100033B963687BB9022000F03AFC3223636091
:100420002B78032B07D163682BB9022000F030FC36
:100430004FF47A73636038BD50220020D103000866
:100440007023002068220020084B187003280CD865
:10045000DFE800F008050208022000F00FBC0220CF
:1004600000F002BC024B00225A6070476822002054
:1004700070230020234B244A10B51C461968013113
:100480003FD004339342F9D16268A24239D31F4B63
:100490009B6803F1006303F580439A4231D2002048
:1004A00000F046FB0220FFF7CFFF194B1A6C002229
:1004B0001A64196E1A66196E596C5A64596E5A6626
:1004C0005A6E5A6942F080025A615A6922F08002DB
:1004D0005A615A691A6942F000521A611A6922F087
:1004E00000521A611B6972B64FF0E0233021C3F845
:1004F000084DD4E9003281F311889D4683F30888C2
:10050000104710BD004000082040000800220020D5
:10051000003802402DE9F04F93B0AA4B0090202202
:10052000FF210AA89D6800F0F3FBA74A1378A3B93E
:10053000A648012103601170302383F311880368FA
:100540000BB101F057FDA24AA04800234FF47A7185
:1005500001F046FD002383F31188009B13B19D4BEE
:10056000009A1A609C4A009C1378032B1EBF00233C
:100570001370984A4FF0000A18BF5360D34656468E
:10058000D146012000F07AFB24B1924B1B68002B6E
:1005900000F01182002000F07DFA0390039B002BF5
:1005A000F2DB012000F060FB039B213B162BE8D817
:1005B00001A252F823F000BF150600083D0600080E
:1005C000D10600088305000883050008830500089C
:1005D0005B0700082B09000845080008A708000869
:1005E000CF080008F508000883050008070900087F
:1005F0008305000879090008B5060008830500088E
:10060000BD09000821060008B5060008830500089A
:10061000A70800080220FFF7C7FE002840F0F58178
:10062000009B0221BAF1000F08BF1C4605A841F249
:100630001233ADF8143000F04BFAA2E74FF47A70A1
:1006400000F028FA071EEBDB0220FFF7ADFE0028C2
:10065000E6D0013F052F00F2DA81DFE807F0030A58
:100660000D10133605230593042105A800F030FA78
:1006700017E054480421F9E758480421F6E75848A0
:100680000421F3E74FF01C08404600F053FA08F14C
:1006900004080590042105A800F01AFAB8F12C0FFF
:1006A000F2D1012000FA07F747EA0B0B5FFA8BFB48
:1006B0004FF0000900F078FB26B10BF00B030B2B79
:1006C00008BF0024FFF778FE5BE746480421CDE72A
:1006D000002EA5D00BF00B030B2BA1D10220FFF7AE
:1006E00063FE074600289BD0012000F021FA02207B
:1006F000FFF7AAFE00261FFA86F8404600F028FA07
:10070000044690B10021404600F032FA013600283C
:10071000F1D1BA46044641F21213022105A8ADF800
:1007200014303E4600F0D4F92BE70120FFF78CFE91
:100730002546244B9B68AB4207D9284600F0FAF9BE
:10074000013040F067810435F3E7234B00251D702D
:10075000204BBA465D603E46ACE7002E3FF460AFEA
:100760000BF00B030B2B7FF45BAF0220FFF76CFE4B
:10077000322000F08FF9B0F10008FFF651AF18F009
:1007800003077FF44DAF0F4A926808EB05039342CD
:100790003FF646AFB8F5807F3FF742AF124B01936B
:1007A000B84523DD4FF47A7000F074F90390039A92
:1007B000002AFFF635AF019B039A03F8012B01379E
:1007C000EDE700BF002200206C2300205022002013
:1007D000D10300087023002068220020042200209A
:1007E000082200200C2200206C220020C820FFF7E5
:1007F000DBFD074600283FF413AF1F2D11D8C5F1CC
:10080000200242450AAB25F0030028BF4246834937
:100810000192184400F056FA019A8048FF2100F036
:1008200077FA4FEAA8037D490193C8F38702284667
:1008300000F076FA064600283FF46DAF019B05EB09
:10084000830537E70220FFF7AFFD00283FF4E8AE4D
:1008500000F0BAF900283FF4E3AE0027B846704B29
:100860009B68BB4218D91F2F11D80A9B01330ED0A9
:1008700027F0030312AA134453F8203C0593404683
:10088000042205A900F0F6FA04378046E7E7384667
:1008900000F050F90590F2E7CDF81480042105A886
:1008A00000F016F906E70023642104A8049300F081
:1008B00005F900287FF4B4AE0220FFF775FD00288B
:1008C0003FF4AEAE049800F067F90590E6E7002328
:1008D000642104A8049300F0F1F800287FF4A0AE8E
:1008E0000220FFF761FD00283FF49AAE049800F063
:1008F00063F9EAE70220FFF757FD00283FF490AEC6
:1009000000F072F9E1E70220FFF74EFD00283FF406
:1009100087AE05A9142000F06DF904210746049064
:1009200004A800F0D5F83946B9E7322000F0B2F853
:10093000071EFFF675AEBB077FF472AE384A9268A9
:1009400007EB090393423FF66BAE0220FFF72CFD45
:1009500000283FF465AE27F003074F44B9453FF444
:10096000A9AE484600F0E6F80421059005A800F07D
:10097000AFF809F10409F1E74FF47A70FFF714FDBD
:1009800000283FF44DAE00F01FF9002844D00A9B28
:1009900001330BD008220AA9002000F0C1F9002879
:1009A0003AD02022FF210AA800F0B2F9FFF704FD97
:1009B0001C4801F059FA13B0BDE8F08F002E3FF447
:1009C0002FAE0BF00B030B2B7FF42AAE0023642118
:1009D00005A8059300F072F8074600287FF420AEC2
:1009E0000220FFF7E1FC804600283FF419AEFFF734
:1009F000E3FC41F2883001F037FA059800F018FA6C
:100A0000464600F0D1F93C46BBE5064652E64FF0BB
:100A1000000905E6BA467EE637467CE66C220020F1
:100A200000220020A08601002DE9F84F4FF47A73D0
:100A3000DFF85880DFF8589006460D4602FB03F7B2
:100A4000002498F900305A1C5FFA84FA01D0A342BE
:100A500012D159F8240003682A46D3F820B0314651
:100A60003B46D847854207D1074B012083F800A0B9
:100A7000BDE8F88F0124E4E7002CFBD04FF4FA70B6
:100A800001F0F2F90020F3E7B82300201022002043
:100A90001422002007B50023024601210DF10700B2
:100AA0008DF80730FFF7C0FF20B19DF8070003B0B5
:100AB0005DF804FB4FF0FF30F9E700000A4608B587
:100AC0000421FFF7B1FF80F00100C0B2404208BD31
:100AD00030B4074B0A461978064B53F82140236877
:100AE000DD69054B0146AC46204630BC604700BF7F
:100AF000B823002014220020A086010070B501F068
:100B0000D3FC094E094D3080002428683388834285
:100B100008D901F0C3FC2B6804440133B4F5804FBD
:100B20002B60F2D370BD00BFBA23002078230020D1
:100B300001F070BD00F1006000F580400068704772
:100B400000F10060920000F5804001F0FBBC000065
:100B5000054B1A68054B1B889B1A834202D9104427
:100B600001F09CBC0020704778230020BA230020AD
:100B700038B5084D044629B128682044BDE83840FE
:100B800001F0ACBC2868204401F090FC0028F3D0B0
:100B900038BD00BF7823002010F003030AD1B0F560
:100BA000047F05D200F10050A0F51040D0F80038C5
:100BB000184670470023FBE700F10050A0F51040F5
:100BC000D0F8100A70470000064991F8243033B17C
:100BD0000023086A81F824300822FFF7B1BF012002
:100BE000704700BF7C230020014B1868704700BF8E
:100BF000002004E070B5194B1D68194B0138C5F38E
:100C00000B0408442D0C04221E88A6420BD15C68FC
:100C10000A46013C824213460FD214F9016F4EB1CD
:100C200002F8016BF6E7013A03F10803ECD18142C7
:100C30000B4602D22C2203F8012B0A4A05241688FF
:100C4000AE4204D1984284BF967803F8016B013C10
:100C500002F10402F3D1581A70BD00BF002004E075
:100C6000503B00083C3B0008022802BF024B4FF4F7
:100C700080529A61704700BF00100240022802BFF4
:100C8000024B4FF080529A61704700BF0010024043
:100C9000022801BF024A536983F4805353617047AD
:100CA0000010024070B504464FF47A764CB1412CE6
:100CB000254628BF412506FB05F001F0D5F8641B49
:100CC000F4E770BD10B50023934203D0CC5CC4544C
:100CD0000133F9E710BD000010B5013810F9013FEC
:100CE0003BB191F900409C4203D11AB10131013A64
:100CF000F4E71AB191F90020981A10BD1046FCE7EC
:100D000003460246D01A12F9011B0029FAD1704796
:100D100002440346934202D003F8011BFAE77047EE
:100D20002DE9F8431F4D144695F8242007468846C0
:100D300052BBDFF870909CB395F824302BB9202279
:100D4000FF2148462F62FFF7E3FF95F82400C0F12A
:100D50000802A24228BF2246D6B24146920005EBC5
:100D60008000FFF7AFFF95F82430A41B1E44F6B2B5
:100D7000082E17449044E4B285F82460DBD1FFF7D5
:100D800023FF0028D7D108E02B6A03EB82038342BC
:100D9000CFD0FFF719FF0028CBD10020BDE8F883A2
:100DA0000120FBE77C230020024B1A78024B1A70CB
:100DB000704700BFB82300201022002038B5174C20
:100DC000174D204600F0B6FB2946204600F0DEFB1A
:100DD0002D686A6D936B23F4002393634FF47A704C
:100DE000FFF760FF0F49284600F0D6FC6A6D0E4DF4
:100DF000936B28680D4943F400239363A0424FF49A
:100E0000E1330B6001D000F0F5FA6868A04204D02D
:100E1000BDE83840054900F0EDBA38BD98280020FB
:100E20005C3C0008643C000814220020A42300203D
:100E300070B50C4B0C4D1E780C4B55F826209A4281
:100E400004460DD00A4B002114221846FFF760FF1C
:100E50000460014655F82600BDE8704000F0CABAAB
:100E600070BD00BFB8230020142200209828002065
:100E7000A423002030B5094D0A4491420DD011F849
:100E8000013B5840082340F30004013B2C4013F081
:100E9000FF0384EA5000F6D1EFE730BD2083B8EDC0
:100EA000026843681143016003B1184770470000AE
:100EB000024AD36843F0C003D36070470044004047
:100EC00010B5054C054A0021204600F071FA044A8D
:100ED000044BC4E9972310BDBC230020B10E0008C9
:100EE0000044004080DE8002234A037C002918BFB2
:100EF0000A46012B30B5C0F868220CD11F4B98422E
:100F000009D11F4B196C41F400311964196E41F479
:100F1000003119661B6EB2F904501468D0F86032C3
:100F2000D0F85C12002D03EB5403B3FBF4F3BEBF07
:100F300023F0070503F0070343EA450394888B6019
:100F4000D38843F040030B61138943F001034B61E5
:100F500044F4045343F02C03CB6004F4A054002366
:100F60000B60B4F5806F0B684B680CBF7F23FF23C9
:100F700080F8643230BD00BF703B0008BC23002005
:100F8000003802402DE9F041D0F85C62F768336820
:100F9000DA0504469DB20DD5302383F311884FF452
:100FA00080610430FFF77CFF6FF4807333600023AF
:100FB00083F31188302383F3118804F1040815F0BA
:100FC0002F033AD183F31188380615D5290613D596
:100FD000302383F3118804F1380000F065F900280C
:100FE0004EDA0821201DFFF75BFF4FF67F733B4071
:100FF000F360002383F311887A0616D56B0614D5A7
:10100000302383F31188D4E913239A420AD1236C45
:1010100043B127F040073F041021201D3F0CFFF78C
:101020003FFFF760002383F31188D4F86822D36868
:1010300043B3BDE8F041106918472B0714D015F0F1
:10104000080F0CBF00214FF48071E80748BF41F042
:101050002001AA0748BF41F040016B0748BF41F09B
:1010600080014046FFF71CFFAD06736805D594F874
:1010700064122046194000F0CBF93568ADB29EE706
:101080007060B6E7BDE8F081F8B51546826806697C
:10109000AA420B46816938BF8568761AB542044674
:1010A0000BD218462A46FFF70DFEA3692B44A36115
:1010B000A3685B1BA3602846F8BD0CD918463246CE
:1010C000FFF700FEAF1BE1683A463044FFF7FAFD38
:1010D000E3683B44EBE718462A46FFF7F3FDE36875
:1010E000E5E7000083689342F7B51546044638BF2C
:1010F0008568D0E90460361AB5420BD22A46FFF75C
:10110000E1FD63692B446361A36828465B1BA36010
:1011100003B0F0BD0DD932460191FFF7D3FD01991F
:10112000E068AF1B3A463144FFF7CCFDE3683B442F
:10113000E9E72A46FFF7C6FDE368E4E710B50A448D
:101140000024C361029B8460C0E90000C0E905116E
:10115000C1600261036210BD08B5D0E90532934257
:1011600001D1826882B98268013282605A1C426170
:101170001970D0E904329A4224BFC3684361002148
:1011800000F08EFE002008BD4FF0FF30FBE70000AE
:1011900070B5302304460E4683F31188A568A5B1C7
:1011A000A368A269013BA360531CA361157822695F
:1011B000934224BFE368A361E3690BB120469847DB
:1011C000002383F31188284607E03146204600F0CB
:1011D00057FE0028E2DA85F3118870BD2DE9F74F3C
:1011E00004460E4617469846D0F81C904FF0300A39
:1011F0008AF311884FF0000B154665B12A46314637
:101200002046FFF741FF034660B94146204600F003
:1012100037FE0028F1D0002383F31188781B03B038
:10122000BDE8F08FB9F1000F03D001902046C84708
:10123000019B8BF31188ED1A1E448AF31188DCE7B9
:10124000C0E90511C160C3611144009B8260C0E91F
:101250000000016103627047F8B504460D4616466A
:10126000302383F31188A768A7B1A368013BA3606B
:1012700063695A1C62611D70D4E904329A4224BF2A
:10128000E3686361E3690BB120469847002080F36F
:10129000118807E03146204600F0F2FD0028E2DA2E
:1012A00087F31188F8BD0000D0E905239A4210B5F4
:1012B00001D182687AB98268013282605A1C8261E7
:1012C0001C7803699A4224BFC3688361002100F03F
:1012D000E7FD204610BD4FF0FF30FBE72DE9F74F4B
:1012E00004460E4617469846D0F81C904FF0300A38
:1012F0008AF311884FF0000B154665B12A46314636
:101300002046FFF7EFFE034660B94146204600F055
:10131000B7FD0028F1D0002383F31188781B03B0B8
:10132000BDE8F08FB9F1000F03D001902046C84707
:10133000019B8BF31188ED1A1E448AF31188DCE7B8
:10134000026843681143016003B118477047000009
:101350001430FFF743BF00004FF0FF331430FFF7A6
:101360003DBF00003830FFF7B9BF00004FF0FF333A
:101370003830FFF7B3BF00001430FFF709BF00009B
:101380004FF0FF311430FFF703BF00003830FFF794
:1013900063BF00004FF0FF323830FFF75DBF000041
:1013A000012914BF6FF0130000207047FFF788BDBC
:1013B00037B515460E4A026000224260C0E902229B
:1013C0000122044602740B46009000F15C014FF4C8
:1013D00080721430FFF7B2FE00942B464FF48072F7
:1013E00004F5AE7104F13800FFF72AFF03B030BDF9
:1013F000843B000810B53023044683F31188FFF7BF
:1014000073FD02232374002080F3118810BD0000B7
:1014100038B5C36904460D461BB904210844FFF7DB
:101420008FFF294604F11400FFF796FE002806DA24
:10143000201D4FF40061BDE83840FFF781BF38BD83
:10144000026843681143016003B118477047000008
:1014500013B5446BD4F894341A681178042915D163
:10146000217C022912D11979128901238B40134260
:101470000CD101A904F14C0001F016FFD4F89444FA
:10148000019B21790246206800F0D0F902B010BD1E
:10149000143001F099BE00004FF0FF33143001F01A
:1014A00093BE00004C3001F06BBF00004FF0FF33E3
:1014B0004C3001F065BF0000143001F067BE000041
:1014C0004FF0FF31143001F061BE00004C3001F0EC
:1014D00037BF00004FF0FF324C3001F031BF000049
:1014E0000020704710B5D0F894341A681178042998
:1014F000044617D1017C022914D15979528901235C
:101500008B4013420ED1143001F0FAFD024648B16F
:10151000D4F894444FF4807361792068BDE810409A
:1015200000F072B910BD0000406BFFF7DBBF000098
:10153000704700007FB5124B036000234360C0E991
:101540000233012502260F4B0574044602900193D5
:1015500000F18402294600964FF48073143001F0A4
:10156000ABFD094B0294CDE9006304F523724FF4FF
:101570008073294604F14C0001F072FE04B070BD86
:10158000AC3B000829150008511400080B683022F4
:1015900082F311880A7903EB820290614A79093259
:1015A00043F822008A7912B103EB82039861022387
:1015B000C0F894140374002080F311887047000071
:1015C00038B5037F044613B190F85430ABB9201DF1
:1015D00001250221FFF734FF04F1140025776FF095
:1015E000010100F069FC84F8545004F14C006FF0E4
:1015F0000101BDE8384000F05FBC38BD10B50121E5
:1016000004460430FFF71CFF0023237784F854308E
:1016100010BD000038B504460025143001F064FD0B
:1016200004F14C00257701F033FE201D84F854505E
:101630000121FFF705FF2046BDE83840FFF752BF04
:1016400090F8443003F06003202B07D190F8452038
:10165000212A4FF0000303D81F2A06D80020704724
:10166000222AFBD1C0E90E3303E0034A826307223A
:10167000C2630364012070471C22002037B5D0F8F4
:1016800094341A681178042904461AD1017C02297D
:1016900017D11979128901238B40134211D100F11E
:1016A0004C05284601F0B4FE58B101A9284601F0C6
:1016B000FBFDD4F89444019B21790246206800F098
:1016C000B5F803B030BD0000F0B500EB810385B084
:1016D0009E6904460D46FEB1302383F3118804EB66
:1016E0008507301D0821FFF7ABFEFB685B691B68AF
:1016F00006F14C001BB1019001F0E4FD019803A933
:1017000001F0D2FD024648B1039B2946204600F075
:101710008DF8002383F3118805B0F0BDFB685A698A
:101720001268002AF5D01B8A013B1340F1D104F165
:101730004402EAE7093138B550F82140DCB13023E2
:1017400083F31188D4F894241368527903EB82034D
:10175000DB689B695D6845B104216018FFF770FE86
:10176000294604F1140001F0D5FC2046FFF7BAFE2B
:10177000002383F3118838BD7047000001F034B8AE
:10178000012303700023C0E90133C3618362036254
:10179000C36243620363704738B50446302383F362
:1017A00011880025C0E90355C0E90555416001F0E5
:1017B0002BF80223237085F31188284638BD0000DA
:1017C00070B500EB810305465069DA600E46144699
:1017D00018B110220021FFF79BFAA06918B110225E
:1017E0000021FFF795FA31462846BDE8704001F028
:1017F000D5B80000826802F0011282600022C0E9C0
:101800000422826101F056B9F0B400EB81044789EB
:10181000E4680125A4698D403D4345812360002390
:10182000A2606360F0BC01F071B90000F0B400EB9D
:1018300081040789E468012564698D403D43058181
:1018400023600023A2606360F0BC01F0EBB90000EC
:1018500070B50223002504460370C0E90255C0E9B3
:101860000455C564856180F8345001F033F863682D
:101870001B6823B129462046BDE87040184770BD5B
:101880000378052B10B504460AD080F850300523A4
:10189000037043681B680BB1042198470023A360C1
:1018A00010BD00000178052906D190F8502043684A
:1018B00002701B6803B118477047000070B590F8BC
:1018C0003430044613B1002380F8343004F144026C
:1018D000204601F011F963689B68B3B994F844306D
:1018E00013F0600535D00021204601F0B1FB002146
:1018F000204601F0A3FB63681B6813B10621204654
:101900009847062384F8343070BD20469847002855
:10191000E4D0B4F84A30E26B9A4288BFE36394F9AA
:101920004430E56B002B4FF0300380F20381002D33
:1019300000F0F280092284F8342083F3118800211A
:10194000D4E90E232046FFF771FF002383F31188AB
:10195000DAE794F8452003F07F0343EA022340F2DC
:101960000232934200F0C58021D8B3F5807F48D081
:101970000DD8012B3FD0022B00F09380002BB2D169
:1019800004F14C02A2630222E2632364C1E7B3F5CF
:10199000817F00F09B80B3F5407FA4D194F846305E
:1019A000012BA0D1B4F84C3043F0020332E0B3F580
:1019B000006F4DD017D8B3F5A06F31D0A3F5C06339
:1019C000012B90D8636894F846205E6894F847101D
:1019D000B4F848302046B047002884D04368A36359
:1019E0000368E3631AE0B3F5106F36D040F60242A5
:1019F00093427FF478AF5C4BA3630223E36300233D
:101A0000C3E794F84630012B7FF46DAFB4F84C3047
:101A100023F00203C4E90E55A4F84C30256478E79E
:101A2000B4F84430B3F5A06F0ED194F8463084F882
:101A30004E30204600F0A6FF63681B6813B10121F9
:101A400020469847032323700023C4E90E339CE704
:101A500004F14F03A3630123C3E72378042B10D1C0
:101A6000302383F311882046FFF7C4FE85F31188E5
:101A70000321636884F84F5021701B680BB1204626
:101A8000984794F84630002BDED084F84F3004237A
:101A9000237063681B68002BD6D00221204698472C
:101AA000D2E794F848301D0603F00F0120460AD50E
:101AB00001F014F8012804D002287FF414AF2B4B56
:101AC0009AE72B4B98E700F0FBFFF3E794F84630DA
:101AD000002B7FF408AF94F8483013F00F01B3D017
:101AE0001A06204602D501F0C7FAADE701F0BAFAAE
:101AF000AAE794F84630002B7FF4F5AE94F848300E
:101B000013F00F01A0D01B06204602D501F0A0FA69
:101B10009AE701F093FA97E7142284F8342083F3CC
:101B200011882B462A4629462046FFF76DFE85F38D
:101B30001188E9E65DB1152284F8342083F3118819
:101B40000021D4E90E232046FFF75EFEFDE60B22BE
:101B500084F8342083F311882B462A4629462046F0
:101B6000FFF764FEE3E700BFDC3B0008D43B00085E
:101B7000D83B000838B590F834300446002B3ED0EE
:101B8000063BDAB20F2A34D80F2B32D8DFE803F045
:101B9000373131082232313131313131313137375A
:101BA000C56BB0F84A309D4214D2C3681B8AB5FB9E
:101BB000F3F203FB12556DB9302383F311882B46E2
:101BC0002A462946FFF732FE85F311880A2384F856
:101BD00034300EE0142384F83430302383F311883A
:101BE00000231A4619462046FFF70EFE002383F312
:101BF000118838BD036C03B198470023E7E7002143
:101C0000204601F025FA0021204601F017FA63680A
:101C10001B6813B10621204698470623D7E700002A
:101C200010B590F83430142B044629D017D8062B61
:101C300005D001D81BB110BD093B022BFBD80021F8
:101C4000204601F005FA0021204601F0F7F963680B
:101C50001B6813B1062120469847062319E0152B6F
:101C6000E9D10B2380F83430302383F3118800232B
:101C70001A461946FFF7DAFD002383F31188DAE7E5
:101C8000C3689B695B68002BD5D1036C03B198478F
:101C9000002384F83430CEE700230375826803699B
:101CA0001B6899689142FBD25A68036042601060D9
:101CB0005860704700230375826803691B68996840
:101CC0009142FBD85A6803604260106058607047C8
:101CD00008B50846302383F311880B7D032B05D00C
:101CE000042B0DD02BB983F3118808BD8B6900221A
:101CF0001A604FF0FF338361FFF7CEFF0023F2E756
:101D0000D1E9003213605A60F3E70000FFF7C4BF67
:101D1000054BD9680875186802681A60536001227B
:101D20000275D860FEF7EEBA2826002030B50C4BBD
:101D3000DD684B1C87B004460FD02B46094A684625
:101D400000F04EF92046FFF7E3FF009B13B1684611
:101D500000F050F9A86907B030BDFFF7D9FFF9E7E7
:101D600028260020D11C0008044B1A68DB68906804
:101D70009B68984294BF00200120704728260020CD
:101D8000084B10B51C68D86822681A60536001229D
:101D90002275DC60FFF78EFF01462046BDE810404B
:101DA000FEF7B0BA2826002038B5074C0749084886
:101DB000012300252370656001F068FB0223237076
:101DC00085F3118838BD00BF90280020E43B00084F
:101DD0002826002000F044B9034A516853685B1A72
:101DE0009842FBD8704700BF001000E08B600223D0
:101DF00008618B82084670478368A3F1840243F828
:101E0000142C026943F8442C426943F8402C094AD7
:101E100043F8242CC26843F8182C022203F80C2C37
:101E2000002203F80B2C044A43F8102CA3F12000E5
:101E3000704700BF1D0300082826002008B5FFF7E3
:101E4000DBFFBDE80840FFF761BF0000024BDB6825
:101E500098610F20FFF75CBF28260020302383F312
:101E60001188FFF7F3BF000008B50146302383F364
:101E700011880820FFF75AFF002383F3118808BD5B
:101E8000064BDB6839B1426818605A6013604360E2
:101E90000420FFF74BBF4FF0FF307047282600208B
:101EA0000368984206D01A6802605060996118462B
:101EB000FFF72CBF7047000038B504460D46206878
:101EC000844200D138BD036823605C608561FFF700
:101ED0001DFFF4E710B503689C68A2420CD85C684B
:101EE0008A600B604C602160596099688A1A9A6018
:101EF0004FF0FF33836010BD1B68121BECE700003E
:101F00000A2938BF0A2170B504460D460A26601911
:101F100001F0B4FA01F09CFA041BA54203D8751C29
:101F20002E460446F3E70A2E04D9BDE8704001208E
:101F300001F0ECBA70BD0000F8B5144B0D46D96144
:101F400003F1100141600A2A1969826038BF0A2230
:101F5000016048601861A818144601F07FFA0A274A
:101F600001F076FA431BA342064606D37C1C2819CF
:101F700001F084FA27463546F2E70A2F04D9BDE876
:101F8000F840012001F0C2BAF8BD00BF28260020A9
:101F9000F8B506460D4601F05BFA0F4A134653F8B2
:101FA000107F9F4206D12A4601463046BDE8F840E0
:101FB000FFF7C2BFD169BB68441A2C1928BF2C4651
:101FC000A34202D92946FFF79BFF22463146034828
:101FD000BDE8F840FFF77EBF282600203826002005
:101FE00010B4C0E9032300235DF8044B4361FFF7FD
:101FF000CFBF000010B5194C236998420DD0D0E92D
:102000000032816813605A609A680A449A6000231B
:1020100003604FF0FF33A36110BD2346026843F80D
:10202000102F53600022026022699A4203D1BDE85A
:10203000104001F01DBA936881680B44936001F071
:1020400007FA2269E1699268441AA242E4D911446C
:10205000BDE81040091AFFF753BF00BF2826002033
:102060002DE9F047DFF8BC8008F110072C4ED8F8B6
:10207000105001F0EDF9D8F81C40AA68031B9A42F1
:102080003ED81444D5E900324FF00009C8F81C408E
:1020900013605A60C5F80090D8F81030B34201D1EF
:1020A00001F0E6F989F31188D5E90331284698470C
:1020B000302383F311886B69002BD8D001F0C8F965
:1020C0006A69A0EB04094A4582460DD2022001F05C
:1020D0001DFA0022D8F81030B34208D151462846E4
:1020E000BDE8F047FFF728BF121A2244F2E712EBCF
:1020F000090938BF4A4629463846FFF7EBFEB5E7DF
:10210000D8F81030B34208D01444211AC8F81C0083
:10211000A960BDE8F047FFF7F3BEBDE8F08700BF58
:10212000382600202826002000207047FEE7000007
:10213000704700004FF0FF307047000002290CD0BC
:10214000032904D00129074818BF00207047032A3B
:1021500005D8054800EBC2007047044870470020CE
:10216000704700BFC03C00082C220020743C0008CF
:1021700070B59AB00546084601A9144600F0C2F8A9
:1021800001A8FEF7BDFD431C5B00C5E90034002239
:10219000237003236370C6B201AB02341046D1B280
:1021A0008E4204F1020401D81AB070BD13F8011B6D
:1021B00004F8021C04F8010C0132F0E708B53023E2
:1021C00083F311880348FFF759FA002383F311883A
:1021D00008BD00BF9828002090F8443003F01F028B
:1021E000012A07D190F845200B2A03D10023C0E92A
:1021F0000E3315E003F06003202B08D1B0F848300F
:102200002BB990F84520212A03D81F2A04D8FFF7BC
:1022100017BA222AEBD0FAE7034A82630722C26385
:1022200003640120704700BF2322002007B5052961
:1022300017D8DFE801F0191603191920302383F3AA
:102240001188104A01900121FFF7BAFA01980E4A4D
:102250000221FFF7B5FA0D48FFF7DCF9002383F3FD
:10226000118803B05DF804FB302383F3118807481D
:10227000FFF7A6F9F2E7302383F311880348FFF74D
:10228000BDF9EBE7143C0008383C00089828002012
:1022900038B50C4D0C4C0D492A4604F10800FFF7E7
:1022A00067FF05F1CA0204F110000949FFF760FF5A
:1022B00005F5CA7204F118000649BDE83840FFF779
:1022C00057BF00BF602D00202C220020F03B0008EB
:1022D000FD3B0008083C000870B5044608460D4662
:1022E000FEF70EFDC6B22046013403780BB918463E
:1022F00070BD32462946FEF7EFFC0028F3D10120DD
:10230000F6E700002DE9F04705460C46FEF7F8FC1D
:102310002B49C6B22846FFF7DFFF08B10736F6B2F1
:1023200028492846FFF7D8FF08B11036F6B2632EC9
:102330000BD8DFF88C80DFF88C90234FDFF894A067
:102340002E7846B92670BDE8F08729462046BDE8BC
:10235000F04701F0D5BB252E2ED107224146284655
:10236000FEF7BAFC70B9194B224603F10C0153F881
:10237000040B42F8040B8B42F9D11B8813800735FC
:102380000E34DDE7082249462846FEF7A5FC98B939
:102390000F4BA21C197809090232C95D02F8041C0E
:1023A00013F8011B01F00F015345C95D02F8031C2E
:1023B000F0D118340835C3E704F8016B0135BFE7E5
:1023C000E03C0008083C0008F73C0008E83C000836
:1023D000107AFF1F1C7AFF1FBFF34F8F024AD3688A
:1023E000DB03FCD4704700BF003C024008B5094B3A
:1023F0001B7873B9FFF7F0FF074B1A69002ABFBFBC
:10240000064A5A6002F188325A601A6822F48062E1
:102410001A6008BDBE2F0020003C02402301674522
:1024200008B50B4B1B7893B9FFF7D6FF094B1A6918
:1024300042F000421A611A6842F480521A601A6827
:1024400022F480521A601A6842F480621A6008BD51
:10245000BE2F0020003C02401728F0B516D80C4CC7
:102460000C4923787BB90C4D0E4618234FF00062BF
:1024700055F8047B46F8042B013B13F0FF033A4464
:10248000F6D10123237051F82000F0BD0020FCE7B5
:1024900020300020C02F0020083D0008014B53F8D9
:1024A00020007047083D000818207047172810B515
:1024B000044601D9002010BDFFF7CEFF064B53F8AC
:1024C00024301844C21A0BB90120F4E71268013213
:1024D000F0D1043BF6E700BF083D0008172838B5E7
:1024E000044628D81549FFF777FFFFF77FFFF3234E
:1024F000CB600C23B0FBF3F203FB1205D30143EADC
:10250000C503DBB243F4007343F002030B610B69B4
:1025100043F480330B61FFF75FFFFFF79DFF084B2C
:1025200053F8241000F0DAF8FFF77AFF2046BDE8F0
:102530003840FFF7BBBF002038BD00BF003C024061
:10254000083D0008F8B512F00103144642D1821884
:10255000B2F1026F57D82D4B1B6813F0010352D014
:102560002B4DFFF743FFF323EB60FFF735FF40F2FE
:102570000127032C15D824F001046618244C401AB6
:1025800040F20117B142236900EB010524D123F089
:1025900001032361FFF744FF0120F8BD043C043030
:1025A000E7E78307E7D12B6923F440732B612B699D
:1025B0003B432B6151F8046B0660BFF34F8FFFF76D
:1025C0000BFF03689E42E9D02B6923F001032B61C6
:1025D000FFF726FF0020E0E723F44073236123691F
:1025E0003B4323610B882B80BFF34F8FFFF7F4FE33
:1025F0002D8831F8023BADB2AB42C3D0236923F042
:1026000001032361E4E71846C7E700BF0038024032
:10261000003C0240084908B50B7828B11BB9FFF708
:10262000E5FE01230B7008BD002BFCD0BDE808407F
:102630000870FFF7F5BE00BFBE2F002010B50244A2
:10264000064BD2B2904200D110BD441C00B253F8E8
:10265000200041F8040BE0B2F4E700BF502800402E
:102660000F4B30B51C6F240407D41C6F44F4007466
:102670001C671C6F44F400441C670A4C236843F435
:10268000807323600244084BD2B2904200D130BD27
:10269000441C00B251F8045B43F82050E0B2F4E768
:1026A00000380240007000405028004007B5012269
:1026B00001A90020FFF7C2FF019803B05DF804FBF9
:1026C00013B50446FFF7F2FFA04205D0012201A98D
:1026D00000200194FFF7C4FF02B010BD7047000056
:1026E000094B5A88B2F5805F10460BD022F00203E6
:1026F00041F20102934205D041F20703C31A584246
:102700005841704701207047002004E0034B1A68CD
:102710001AB9034AD2F874281A607047243000208E
:102720000030024008B5FFF7F1FF024B1868C0F314
:10273000407008BD2430002070470000FEE7000014
:102740000A4B0B480B4A90420BD30B4BDA1C121A64
:10275000C11E22F003028B4238BF00220021FEF787
:10276000D7BA53F8041B40F8041BECE7EC3E000812
:1027700020310020203100202031002070B5D0E928
:1027800015439E6800224FF0FF3504EB42135101C0
:10279000D3F800090028BEBFD3F8000940F08040FC
:1027A000C3F80009D3F8000B0028BEBFD3F8000B14
:1027B00040F08040C3F8000B013263189642C3F822
:1027C0000859C3F8085BE0D24FF00113C4F81C3875
:1027D00070BD0000890141F02001016103699B0681
:1027E000FCD41220FFF7F8BA10B5054C2046FEF7CE
:1027F000C7FF4FF0A0436365024BA36510BD00BF48
:10280000283000208C3D000870B50378012B054668
:1028100050D12A4B446D98421BD1294B5A6B42F040
:1028200080025A635A6D42F080025A655A6D5A69A5
:1028300042F080025A615A6922F080025A610E21E8
:1028400043205B6900F022FC1E4BE3601E4BC4F882
:1028500000380023C4F8003EC02323606E6D4FF49F
:102860005023A3633369002BFCDA012333610C206E
:10287000FFF7B2FA3369DB07FCD41220FFF7ACFA9A
:102880003369002BFCDA0026A6602846FFF776FFA6
:102890006B68C4F81068DB68C4F81468C4F81C6876
:1028A0004BB90A4BA3614FF0FF336361A36843F058
:1028B0000103A36070BD064BF4E700BF2830002081
:1028C000003802404014004003002002003C30C0A9
:1028D000083C30C0F8B5446D054600212046FFF79E
:1028E00079FFA96D00234FF001128F68C4F83438C6
:1028F0004FF00066C4F81C284FF0FF3004EB431281
:1029000001339F42C2F80069C2F8006BC2F808099F
:10291000C2F8080BF2D20B686A6DEB656362102394
:102920001361166916F01006FBD11220FFF754FA56
:10293000D4F8003823F4FE63C4F80038A36943F4E4
:10294000402343F01003A3610923C4F81038C4F8EE
:1029500014380A4BEB604FF0C043C4F8103B084BEF
:10296000C4F8003BC4F81069C4F80039EB6D03F1FA
:10297000100243F48013EA65A362F8BD683D0008C5
:1029800040800010426D90F84E10D2F8003823F4C9
:10299000FE6343EA0113C2F8003870472DE9F8439B
:1029A00000EB8103456DDA68166806F00306731EB6
:1029B000022B05EB41130C4680460FFA81F94FEAD2
:1029C00041104FF00001C3F8101B4FF0010104F15A
:1029D000100398BFB60401FA03F391698EBF334E1A
:1029E00006F1805606F5004600293AD0578A04F1D0
:1029F0005801490137436F50D5F81C180B43C5F8EF
:102A00001C382B180021C3F8101953690127611EC7
:102A1000A7409BB3138A928B9B08012A88BF53431C
:102A2000D8F85C20981842EA034301F1400205EB14
:102A30008202C8F85C00214653602846FFF7CAFEB0
:102A400008EB8900C3681B8A43EA84534834640155
:102A50001E432E51D5F81C381F43C5F81C78BDE81D
:102A6000F88305EB4917D7F8001B21F40041C7F89C
:102A7000001BD5F81C1821EA0303C0E704F13F034B
:102A800005EB83030A4A5A6028462146FFF7A2FE57
:102A900005EB4910D0F8003923F40043C0F80039A1
:102AA000D5F81C3823EA0707D7E700BF00800010DD
:102AB00000040002826D1268C265FFF75FBE00006D
:102AC0005831436D49015B5813F4004004D013F4AE
:102AD000001F0CBF02200120704700004831436DE9
:102AE00049015B5813F4004004D013F4001F0CBFDD
:102AF000022001207047000000EB8101CB68196AB9
:102B00000B6813604B6853607047000000EB810353
:102B100030B5DD68AA691368D36019B9402B84BF4A
:102B2000402313606B8A1468426D1C44013CB4FB63
:102B3000F3F46343033323F0030302EB411043EA4E
:102B4000C44343F0C043C0F8103B2B6803F00303B9
:102B5000012B09B20ED1D2F8083802EB411013F460
:102B6000807FD0F8003B14BF43F0805343F0005304
:102B7000C0F8003B02EB4112D2F8003B43F00443A3
:102B8000C2F8003B30BD00002DE9F041244D6E6DD0
:102B900006EB40130446D3F8087BC3F8087B3807DC
:102BA0000AD5D6F81438190706D505EB8403214653
:102BB000DB6828465B689847FA071FD5D6F81438B3
:102BC000DB071BD505EB8403D968CCB98B69488A30
:102BD0005A68B2FBF0F600FB16228AB91868DA6868
:102BE00090420DD2121AC3E90024302383F31188D6
:102BF0000B482146FFF78AFF84F31188BDE8F08176
:102C0000012303FA04F26B8923EA02036B81CB6888
:102C1000002BF3D021460248BDE8F041184700BF21
:102C20002830002000EB810370B5DD68436D6C69CE
:102C30002668E6604A0156BB1A444FF40020C2F8E9
:102C400010092A6802F00302012A0AB20ED1D3F851
:102C5000080803EB421410F4807FD4F8000914BF75
:102C600040F0805040F00050C4F8000903EB4212DD
:102C7000D2F8000940F00440C2F80009D3F8340843
:102C8000012202FA01F10143C3F8341870BD19B9E9
:102C9000402E84BF4020206020682E8A8419013C89
:102CA000B4FBF6F440EAC44040F000501A44C6E7D2
:102CB0002DE9F8433B4D6E6D06EB40130446D3F807
:102CC0000889C3F8088918F0010F4FEA40171AD095
:102CD000D6F81038DB0716D505EB8003D9684B69A9
:102CE0001868DA68904230D2121A4FF000091A6060
:102CF000C3F80490302383F3118821462846FFF758
:102D000091FF89F3118818F0800F1CD0D6F8343861
:102D10000126A640334216D005EB84036D6DD3F82F
:102D20000CC0DCF814200134E4B2D2F800E005EB6A
:102D300004342F445168714515D3D5F8343823EA4B
:102D40000606C5F83468BDE8F883012303FA04F2E7
:102D50002B8923EA02032B818B68002BD3D02146D9
:102D600028469847CFE7BCF81000AEEB010383423A
:102D700028BF0346D7F8180980B2B3EB800FE2D81A
:102D80009068A0F1040959F8048FC4F80080A0EB02
:102D900009089844B8F1040FF5D818440B44906022
:102DA0005360C7E7283000202DE9F74FA24C656D2E
:102DB0006E69AB691E4016F480586E6107D02046DC
:102DC000FEF746FD03B0BDE8F04F00F04DBC002E0D
:102DD00012DAD5F8003E98489B071EBFD5F8003E92
:102DE00023F00303C5F8003ED5F8043823F00103AF
:102DF000C5F80438FEF756FD370505D58E48FFF7B0
:102E0000BDFC8D48FEF73CFDB0040CD5D5F8083864
:102E100013F0060FEB6823F470530CBF43F4105308
:102E200043F4A053EB6031071BD56368DB681BB923
:102E3000AB6923F00803AB612378052B0CD1D5F8DF
:102E4000003E7D489A071EBFD5F8003E23F00303DD
:102E5000C5F8003EFEF726FD6368DB680BB17648D7
:102E60009847F30274D4B70227D5D4F85490DFF80A
:102E7000C8B100274FF0010A09EB4712D2F8003B16
:102E800003F44023B3F5802F11D1D2F8003B002B7F
:102E90000DDA62890AFA07F322EA0303638104EB7D
:102EA0008703DB68DB6813B1394658469847A36D42
:102EB00001379B68FFB29F42DED9F00617D5676DD8
:102EC0003A6AC2F30A1002F00F0302F4F012B2F5EC
:102ED000802F00F08580B2F5402F08D104EB8303EA
:102EE0000022DB681B6A07F5805790426AD13003E5
:102EF000D5F8184813D5E10302D50020FFF744FEAA
:102F0000A20302D50120FFF73FFE630302D5022092
:102F1000FFF73AFE270302D50320FFF735FE7503BE
:102F20007FF550AFE00702D50020FFF7C1FEA107F3
:102F300002D50120FFF7BCFE620702D50220FFF791
:102F4000B7FE23077FF53EAF0320FFF7B1FE39E759
:102F5000636DDFF8E4A0019300274FF00109A36D32
:102F60009B685FFA87FB9B453FF67DAF019B03EBB8
:102F70004B13D3F8001901F44021B1F5802F1FD174
:102F8000D3F8001900291BDAD3F8001941F0904159
:102F9000C3F80019D3F800190029FBDB5946606D0E
:102FA000FFF718FC218909FA0BF321EA03032381B7
:102FB00004EB8B03DB689B6813B159465046984776
:102FC0000137CCE7910708BFD7F80080072A98BFE0
:102FD00003F8018B02F1010298BF4FEA182884E739
:102FE000023304EB830207F580575268D2F818C009
:102FF000DCF80820DCE9001CA1EB0C0C0021884265
:103000000AD104EB830463689B699A6802449A605E
:103010005A6802445A606AE711F0030F08BFD7F8F4
:1030200000808C4588BF02F8018B01F1010188BF47
:103030004FEA1828E3E700BF28300020436D03EB78
:103040004111D1F8003B43F40013C1F8003B704735
:10305000436D03EB4111D1F8003943F40013C1F87B
:1030600000397047436D03EB4111D1F8003B23F465
:103070000013C1F8003B7047436D03EB4111D1F8D9
:10308000003923F40013C1F80039704700F16043A0
:1030900003F561430901C9B283F80013012200F06E
:1030A0001F039A4043099B0003F1604303F561430A
:1030B000C3F880211A60704730B5039C0172043355
:1030C00004FB0325C0E90653049B03630021059B11
:1030D000C160C0E90000C0E90422C0E90842C0E9BB
:1030E0000A11436330BD0000416A0022C0E90411A7
:1030F000C0E90A22C2606FF00101FEF7DDBE0000E8
:10310000D0E90432934201D1C2680AB9181D704750
:103110000020704703691960C2680132C260C26949
:10312000134482690361934224BF436A036100210F
:10313000FEF7B6BE38B504460D46E3683BB162699A
:10314000131D1268A3621344E362002007E0237A90
:1031500033B929462046FEF793FE0028EDDA38BD44
:103160006FF00100FBE70000C368C269013BC36068
:103170004369134482694361934224BF436A4361B4
:1031800000238362036B03B11847704770B5302387
:10319000044683F31188866A3EB9FFF7CBFF0546E4
:1031A00018B186F31188284670BDA36AE26A13F845
:1031B000015BA362934202D32046FFF7D5FF0023B1
:1031C00083F31188EFE700002DE9F84F04460E461F
:1031D000174698464FF0300989F311880025AA4612
:1031E000D4F828B0BBF1000F09D141462046FFF7C3
:1031F000A1FF20B18BF311882846BDE8F88FD4E9F0
:103200000A12A7EB050B521A934528BF9346BBF150
:10321000400F1BD9334601F1400251F8040B43F82B
:10322000040B9142F9D1A36A40334036A362403582
:10323000D4E90A239A4202D32046FFF795FF8AF386
:103240001188BD42D8D289F31188C9E730465A4661
:10325000FDF738FDA36A5B445E44A3625D44E7E783
:1032600010B5029C0172043303FB0421C0E906136C
:103270000023C0E90A33039B0363049BC460C0E9D5
:103280000000C0E90422C0E90842436310BD000009
:10329000026AC260426AC0E904220022C0E90A222E
:1032A0006FF00101FEF708BED0E904239A4201D174
:1032B000C26822B9184650F8043B0B6070470023DF
:1032C0001846FAE7C368C2690133C360436913440F
:1032D00082694361934224BF436A43610021FEF740
:1032E000DFBD000038B504460D46E3683BB12369F5
:1032F0001A1DA262E2691344E362002007E0237A08
:1033000033B929462046FEF7BBFD0028EDDA38BD6B
:103310006FF00100FBE7000003691960C268013A21
:10332000C260C269134482690361934224BF436A45
:10333000036100238362036B03B1184770470000E9
:1033400070B530230D460446114683F31188866A12
:103350002EB9FFF7C7FF10B186F3118870BDA36ABD
:103360001D70A36AE26A01339342A36204D3E16948
:1033700020460439FFF7D0FF002080F31188EDE7E5
:103380002DE9F84F04460D46904699464FF0300A15
:103390008AF311880026B346A76A4FB949462046EA
:1033A000FFF7A0FF20B187F311883046BDE8F88F02
:1033B000D4E90A073A1AA8EB0607974228BF17462E
:1033C000402F1BD905F1400355F8042B40F8042B7E
:1033D0009D42F9D1A36A4033A3624036D4E90A235F
:1033E0009A4204D3E16920460439FFF795FF8BF335
:1033F00011884645D9D28AF31188CDE729463A4645
:10340000FDF760FCA36A3B443D44A3623E44E5E70C
:10341000D0E904239A4217D1C3689BB1836A8BB168
:10342000043B9B1A0ED01360C368013BC360C369A1
:103430001A44836902619A4224BF436A03610023EC
:1034400083620123184670470023FBE700F036B97A
:10345000014B586A704700BF000C0040034B00222C
:1034600058631A610222DA60704700BF000C004006
:10347000014B0022DA607047000C0040014B58639A
:10348000704700BF000C0040FEE7000070B51B4B0A
:1034900001630025044686B0586085620E4600F040
:1034A000BFF804F11003C4E904334FF0FF33C4E95B
:1034B0000635C4E90044A560E562FFF7C9FF2B4665
:1034C0000246C4E9082304F134010D4A256580232E
:1034D0002046FEF78BFC0123E0600A4A0375009248
:1034E00072680192B268CDE90223074B6846CDE9C4
:1034F0000435FEF7A3FC06B070BD00BF9028002085
:10350000983D00089D3D000889340008024AD36AAE
:103510001843D062704700BF282600204B684360E4
:103520008B688360CB68C3600B6943614B6903623E
:103530008B6943620B6803607047000008B5264B37
:1035400026481A6940F2FF110A431A611A6922F4E7
:10355000FF7222F001021A611A691A6B0A431A6398
:103560001A6D0A431A651E4A1B6D1146FFF7D6FFF6
:1035700002F11C0100F58060FFF7D0FF02F1380175
:1035800000F58060FFF7CAFF02F1540100F580608A
:10359000FFF7C4FF02F1700100F58060FFF7BEFF86
:1035A00002F18C0100F58060FFF7B8FF02F1A8017D
:1035B00000F58060FFF7B2FF02F1C40100F5806002
:1035C000FFF7ACFF02F1E00100F58060FFF7A6FF16
:1035D000BDE8084000F0F0B80038024000000240AA
:1035E000A43D000808B500F06BFAFEF7DDFBFFF71D
:1035F0008DF8BDE80840FEF74BBE000070470000A4
:10360000EFF3098305494A6B22F001024A636833EC
:1036100083F30988002383F31188704700EF00E0EB
:10362000302080F3118862B60C4B0D4AD96821F422
:10363000E0610904090C0A43DA60D3F8FC20094967
:1036400042F08072C3F8FC200A6842F001020A606E
:103650002022DA7783F82200704700BF00ED00E0F7
:103660000003FA05001000E010B5302383F3118841
:103670000E4B5B6813F4006314D0F1EE103AEFF3D5
:103680000984683C4FF08073E361094BDB6B236670
:1036900084F30988FEF768FB10B1064BA36110BDE7
:1036A000054BFBE783F31188F9E700BF00ED00E06D
:1036B00000EF00E02F030008320300080E4B1A6CE5
:1036C00042F008021A641A6E42F008021A660B4AA7
:1036D0001B6E936843F008039360094B53229A6270
:1036E0004FF0FF32DA6200229A615A63DA605A6060
:1036F00001225A611A60704700380240002004E03D
:10370000000C0040094A08B51169D3680B40D9B2D2
:10371000C9439B07116107D5302383F31188FEF756
:1037200059FB002383F3118808BD00BF000C004043
:103730001F4B1A696FEAC2526FEAD2521A611A69B4
:10374000C2F308021A614FF0FF301A695A695861D2
:1037500000215A6959615A691A6A62F080521A62E4
:103760001A6A02F080521A621A6A5A6A58625A6ACF
:1037700059625A6A1A6C42F080521A641A6E42F008
:1037800080521A661A6E0B4A106840F480701060FE
:10379000186F00F44070B0F5007F1EBF4FF480300A
:1037A00018671967536823F40073536000F060B919
:1037B0000038024000700040344B4FF080521A64D1
:1037C000334A4FF4404111601A6842F001021A6016
:1037D0001A689107FCD59A6822F003029A602B4B75
:1037E0009A6812F00C02FBD1196801F0F901196016
:1037F0009A601A6842F480321A601A689203FCD503
:103800005A6F42F001025A67204B5A6F9007FCD55D
:10381000204A5A601A6842F080721A601C4A536843
:103820005904FCD5194B1A689201FCD51A4A9A60C2
:103830000322C3F88C20194B1A68194B9A42194B72
:1038400021D1194A1168194A91421CD140F205123E
:103850001A60144A136803F00F03052BFAD10B4BBF
:103860009A6842F002029A609A6802F00C02082AF2
:10387000FAD15A6C42F480425A645A6E42F4804241
:103880005A665B6E704740F20572E1E7003802400D
:10389000007000401854400700948838002004E06D
:1038A00011640020003C024000ED00E041C20F41E5
:1038B000074A08B5536903F00103536123B1054A70
:1038C00013680BB150689847BDE80840FFF7CCBEBD
:1038D000003C0140A0300020074A08B5536903F0BE
:1038E0000203536123B1054A93680BB1D06898472E
:1038F000BDE80840FFF7B8BE003C0140A030002002
:10390000074A08B5536903F00403536123B1054A1C
:1039100013690BB150699847BDE80840FFF7A4BE92
:10392000003C0140A0300020074A08B5536903F06D
:103930000803536123B1054A93690BB1D0699847D5
:10394000BDE80840FFF790BE003C0140A0300020D9
:10395000074A08B5536903F01003536123B1054AC0
:10396000136A0BB1506A9847BDE80840FFF77CBE68
:10397000003C0140A0300020164B10B55C6904F4F7
:1039800078725A61A30604D5134A936A0BB1D06AC0
:103990009847600604D5104A136B0BB1506B9847DB
:1039A000210604D50C4A936B0BB1D06B9847E20506
:1039B00004D5094A136C0BB1506C9847A30504D584
:1039C000054A936C0BB1D06C9847BDE81040FFF7E7
:1039D0004BBE00BF003C0140A0300020194B10B589
:1039E0005C6904F47C425A61620504D5164A136D81
:1039F0000BB1506D9847230504D5134A936D0BB155
:103A0000D06D9847E00404D50F4A136E0BB1506E89
:103A10009847A10404D50C4A936E0BB1D06E984719
:103A2000620404D5084A136F0BB1506F9847230402
:103A300004D5054A936F0BB1D06F9847BDE810408D
:103A4000FFF712BE003C0140A030002008B503483B
:103A5000FDF798FABDE80840FFF706BEBC2300203A
:103A600008B5FFF74FFEBDE80840FFF7FDBD0000B9
:103A7000062108B50846FFF709FB06210720FFF7D6
:103A800005FB06210820FFF701FB06210920FFF7AF
:103A9000FDFA06210A20FFF7F9FA06211720FFF7A1
:103AA000F5FA06212820FFF7F1FA07213220FFF767
:103AB000EDFABDE808400C212620FFF7E7BA000028
:103AC00008B5FFF735FE00F00DF8FDF76FFCFDF7C8
:103AD00055FEFDF72DFDFFF791FDBDE80840FFF70E
:103AE000B5BC00000023054A19460133102BC2E97A
:103AF000001102F10802F8D1704700BFA030002089
:103B0000034611F8012B03F8012B002AF9D1704765
:103B100053544D3332463F3F3F0053544D333246AA
:103B20003430780053544D33324634327800535495
:103B30004D333246343436585800000001203300EB
:103B40000010410001105A00031059000710310005
:103B500000000000103B0008130400001A3B00089E
:103B600019040000243B0008210400002E3B00083B
:103B700000960000000000000000000000000000AF
:103B800000000000000000006D1300085913000839
:103B900095130008811300088D130008791300089D
:103BA0006513000851130008A1130008000000006D
:103BB000AD14000899140008D5140008C1140008B9
:103BC000CD140008B9140008A514000891140008C9
:103BD000E1140008000000000100000000000000E7
:103BE00063300000E03B0008802600209028002081
:103BF0004865782F50726F6669434E430025424FE7
:103C0000415244252D424C002553455249414C25F3
:103C1000000000000200000000000000C9160008BB
:103C20003517000840004000302D0020402D0020B6
:103C3000020000000000000003000000000000007F
:103C4000791700080000000010000000502D00202F
:103C500000000000010000000000000028300020EB
:103C6000010102002D2200083D210008D921000891
:103C7000BD210008430000007C3C0008090243000D
:103C8000020100C032090400000102020100052403
:103C9000001001052401000104240202052406008D
:103CA00001070582030800FF09040100020A000061
:103CB00000070501024000000705810240000000E6
:103CC00012000000C83C0008120110010200004070
:103CD000AE2D0110000201020301000004030904DB
:103CE00025424F4152442500437562654772656520
:103CF0006E2D736F6C6F0030313233343536373898
:103D00003941424344454600004000000040000065
:103D10000040000000400000000001000000020020
:103D2000000002000000020000000200000002008B
:103D300000000200000002000040000000400000FF
:103D400000400000004000000000010000000200F0
:103D5000000002000000020000000200000002005B
:103D6000000002000000020000000000BD18000872
:103D7000751B0008211C000840004000883000200E
:103D800088300020010000009830002080000000F2
:103D900040010000030000006D61696E0069646C01
:103DA000650000000000812A00020000AAAAAAAA59
:103DB00000000024FFFF00000000000000A00A0037
:103DC0000000000000000000AAAAAAAA000000004B
:103DD000FFFF00000000000000000000140000547D
:103DE00000000000AAAAAAAA14000054FFFF0000C5
:103DF00000000000000000008069100000000000CA
:103E0000AAAA8AAA40561000FFFF0000007070079F
:103E1000000000004001000100000000AAAAAAAAB8
:103E200000010000F7FF000000000000000000009B
:103E30000000000000000000AAAAAAAA00000000DA
:103E4000FFFF000000000000000000000000000074
:103E500000000000AAAAAAAA00000000FFFF0000BC
:103E60000000000000000000000000000000000052
:103E70000A00000000000000030000000000000035
:103E80000000000000000000000000000000000032
:103E90000000000000000000000000000000000022
:103EA000090000000000000000C01F00000000002A
:103EB000FF00000098280020BC230020009600008E
:103EC0000000080096000000000800000400000048
:103ED000DC3C0008000000000000000000000000C2
:0C3EE000000000000000000000000000D6
:00000001FF
